:100000000C9475060C94BC060C94BC060C94BC06AF
:100010000C94BC060C94BC060C94BC060C94BC0658
:100020000C94BC060C94BC060C94A1150C9473168D
:100030000C9474240C94BC060C94BC060C94BC0662
:100040000C94BC060C94BC060C94BC060C94BC0628
:100050000C94BC060C9414250C94BC060C94BC06A1
:100060000C94BC060C9418090C94BC060C94BC06A9
:100070000C94BC060C94BC060C94BC060C94BC06F8
:100080000C94BC060C94BC060C94BC060C94BC06E8
:100090000C94BC060C94BC060C94BC060C94BC06D8
:1000A0000C94BC060C94BC060C94BC06440E480E82
:1000B0004C0E500E540E580E5C0E600E640E680E00
:1000C0006C0E700E740E780E7C0E800E840E880EF0
:1000D0008C0E900E940E980E9C0EA00EA40EA80EE0
:1000E000AC0EB00EB40EB80EBC0EC00EC40EC80ED0
:1000F000CC0ED00E100F420ED40ED60ED80EDA0E45
:10010000DE0EE20EE60EEA0EEF0EF40EF80EFC0E18
:10011000000F040F080F0E0F0E0F0E0F0E0F0E0F15
:100120000E0F0E0F0E0F0E0F0E0F0E0F0E0F0E0FE7
:100130000E0F0E0F0E0F0E0F0E0F0E0F0C0FE01600
:100140000217F0170217F01747176A17F017BF17B3
:10015000D217E91AE91A171B171B741BB21BCB1D08
:10016000CB1DCB1BCB1DCC1CCC1C9F1DCB1DCB1D7D
:10017000B61D8080352B78793980808021087706FC
:1001800007808080201A7A1B168080801E8029803C
:10019000808080808080808080808080221580198F
:1001A000098080801F147B1D0480808023172C050C
:1001B0000A808080260C00360E80808025187610FC
:1001C0000D808080241C80110B80808027127E3758
:1001D0000F8080802A804F7D28808080743051522B
:1001E000328080802D137C38338080802E2F507594
:1001F000348025630025730D0A00522C310D0A004E
:1002000053592C464646340D0A0053482C3030339F
:10021000430D0A00537E2C360D0A0053572C3830FC
:1002200030300D0A00534D2C340D0A0053532C4B23
:100230006579626F6172642F4D6F7573650D0A0089
:10024000532D2C546D6B42540D0A0053462C310D26
:100250000A002D2D2D0D0A0045786974696E6720FE
:10026000636F6E666967206D6F6465202E2E2E0A9F
:10027000002B0D0A00760D0A0024242400456E741C
:100280006572696E6720636F6E666967206D6F6463
:1002900065202E2E2E0A00522C310D0A0053522CAE
:1002A0005A0D0A00555342206D6F64650A0041756E
:1002B000746F206D6F64650A00253032750A002561
:1002C0003032753A00253032753A004241543A20B6
:1002D00025756D560900757074696D653A20253075
:1002E000327520253032753A253032753A25303254
:1002F000750A00564255533A2025580A0052656D3A
:100300006F746557616B657570456E61626C65648D
:100310003A2025580A000A003F004C4F5700444934
:10032000534348470043484152470046554C4C0010
:10033000626174746572793A200055534220537497
:100340006174653A2025730A00636F6E6669675FA2
:100350006D6F64653A2025580A00726E34325F6111
:1003600075746F636F6E6E656374696E6728293A82
:100370002025580A00726E34323A2025730A00662E
:100380006F7263655F7573623A2025580A00707258
:100390006F746F636F6C3A2025730A000A2D2D2D40
:1003A0002D2D20524E2D343220696E666F202D2D5A
:1003B0002D2D2D0A00753A20202020202020746F3A
:1003C00067676C6520466F72636520555342206DE8
:1003D0006F64650A00703A20202020202020706180
:1003E0006972696E670A00536C636B3A20202020A3
:1003F000524E2D343220696E697469616C697A6578
:100400000A0044656C3A2020202020656E746572D5
:100410002F6578697420524E2D343220636F6E66DA
:100420006967206D6F64650A00623A2020202020F1
:1004300020206261747465727920766F6C746167D4
:10044000650A00693A20202020202020524E2D34B9
:100450003220696E666F0A000A0A2D2D2D2D2D207F
:10046000426C7565746F6F746820524E2D34322063
:1004700048656C70202D2D2D2D2D0A0025303275EC
:100480003A253032753A253032750925756D560A90
:10049000004C4544207374617475733A20253032E2
:1004A000580A002025303258002563005B735D0038
:1004B0004B6579626F6172642073746172740A00B3
:1004C000524E2D343220696E69740A000A55534227
:1004D00020696E69740A005B445D005B435D001235
:1004E00003480048004B00420020006D006F00648C
:1004F0000000000E0374002E006D002E006B002E15
:100500000000000403090409027400040100A03281
:100510000904000001030101000921110100012269
:1005200040000705810308000A09040100010301D6
:100530000200092111010001224D00070582030874
:10054000000A090402000103000000092111010052
:10055000012236000705830308000A09040300028C
:100560000300000009211101000122220007058477
:1005700003200001070504032000011201100100FF
:10058000000008EDFE42420401010200010631FFB5
:100590000974A1010975150026FF009520750881D1
:1005A000020976150026FF00952075089102C00506
:1005B000010980A101850216810026B7001A810079
:1005C0002AB700751095018100C0050C0901A10131
:1005D0008503160100269C021A01002A9C02751050
:1005E00095018100C005010902A1010901A10005D1
:1005F0000919012905150025019505750181029547
:1006000001750381010501093009311581257F95A7
:10061000027508810609381581257F9501750881C5
:1006200006050C0A38021581257F9501750881069B
:10063000C0C005010906A101050719E029E7150059
:10064000250195087501810295017508810105084C
:10065000190129059505750191029501750391010F
:100660000507190029FF150026FF0095067508816A
:1006700000C0636F6E73756D65723A202530345813
:100680000A0073797374656D3A20253034580A0076
:100690000A002530325820006B6579626F61726400
:1006A0003A20004C45443A20253032580A00253083
:1006B00032583A202530386225730A00722F6320A1
:1006C00030313233343536370A004F6E6573686F18
:1006D000743A2074696D656F75740A00290A0025E3
:1006E00075002F002575005D280025640020002579
:1006F0006400200025640020002564007C00253073
:100700003258006D6F7573656B6579205B62746E2E
:100710007C782079207620685D287265702F61636F
:100720006C293A205B006D6B5F776865656C5F7460
:10073000696D655F746F5F6D6178203D2025640A87
:10074000006D6B5F776865656C5F6D61785F737076
:10075000656564203D2025640A006D6B5F74696DDA
:10076000655F746F5F6D6178203D2025640A006DC0
:100770006B5F6D61785F7370656564203D202564F3
:100780000A006D6B5F696E74657276616C203D2046
:1007900025640A006D6B5F64656C6179203D2025DE
:1007A000640A006D6B5F776865656C5F74696D6581
:1007B0005F746F5F6D6178203D2025640A006D6B6A
:1007C0005F776865656C5F6D61785F7370656564A0
:1007D000203D2025640A006D6B5F74696D655F7450
:1007E0006F5F6D6178203D2025640A006D6B5F6D41
:1007F00061785F7370656564203D2025640A006D33
:100800006B5F696E74657276616C203D2025640AA9
:10081000006D6B5F64656C6179203D2025640A0082
:100820000A00257500363A20776865656C5F746943
:100830006D655F746F5F6D61783A20000A00257501
:1008400000353A20776865656C5F6D61785F73701D
:100850006565643A20000A00257500343A20746901
:100860006D655F746F5F6D61783A20000A002575D1
:1008700000333A206D61785F73706565643A2000DB
:100880000A00257500323A20696E74657276616CD3
:10089000286D73293A20000A00257500313A20643A
:1008A000656C6179282A31306D73293A20000A0974
:1008B0002D2056616C756573202D0A004D3E004D4C
:1008C00025643E20003F0073657420646566617591
:1008D0006C740A00433E2000776865726520646589
:1008E0006C74613A20637572736F723D25642C20BD
:1008F000776865656C3D25640A5365652068747486
:10090000703A2F2F656E2E77696B69706564696127
:100910002E6F72672F77696B692F4D6F7573655FE7
:100920006B6579730A000A092D204D6F7573656B2D
:100930006579202D0A4553432F713A097175697401
:100940000A313A0964656C6179282A31306D73295E
:100950000A323A09696E74657276616C286D732982
:100960000A333A096D61785F73706565640A343AD9
:100970000974696D655F746F5F6D61780A353A0956
:10098000776865656C5F6D61785F73706565640A33
:10099000363A09776865656C5F74696D655F746F79
:1009A0005F6D61780A0A703A097072696E74207618
:1009B000616C7565730A643A0973657420646566D1
:1009C00061756C74730A75703A092B310A646F771C
:1009D0006E3A092D310A706775703A092B31300A69
:1009E0007067646F776E3A092D31300A0A7370654B
:1009F0006564203D2064656C7461202A206D6178F7
:100A00005F7370656564202A202872657065617463
:100A1000202F2074696D655F746F5F6D6178290A9E
:100A2000003F004D3E2000433E20004C25640A005C
:100A30000A092D20436F6E736F6C65202D0A455394
:100A4000432F713A09717569740A6D3A096D6F75B2
:100A500073656B65790A000A092D204D616769632A
:100A6000202D0A643A0964656275670A783A096458
:100A700065627567206D61747269780A6B3A096402
:100A800065627567206B6579626F6172640A6D3AA1
:100A9000096465627567206D6F7573650A763A093A
:100AA00076657273696F6E0A733A0973746174754F
:100AB000730A633A09636F6E736F6C65206D6F64C0
:100AC000650A302D343A096C61796572302D34280D
:100AD0004631302D4634290A506175733A09626FE8
:100AE0006F746C6F616465720A003F0074696D65B4
:100AF000725F72656164333228293A202530346C84
:100B0000580A006B6579626F6172645F69646C6535
:100B10003A2025580A006B6579626F6172645F70D4
:100B2000726F746F636F6C3A2025580A00686F7398
:100B3000745F6B6579626F6172645F6C6564732862
:100B4000293A2025580A000A092D2053746174752A
:100B500073202D0A004743433A20342E392E322089
:100B60004156522D4C4942433A20312E382E307393
:100B7000766E204156525F415243483A2061767268
:100B8000350A004F5054494F4E533A204C55464178
:100B9000204D4F5553454B45592045585452414BD4
:100BA000455920434F4E534F4C4520434F4D4D41E7
:100BB0004E44204B45594D41505F53454354494F96
:100BC0004E20343039360A004255494C443A2035DB
:100BD0003732633236352D646972747920283134A6
:100BE0003A33303A3337204A616E20323520323082
:100BF0003137290A005649443A2030784645454461
:100C000028742E6D2E6B2E29205049443A203078BE
:100C1000343234322848484B42206D6F64292056C4
:100C200045523A203078303130340A00444553433D
:100C30003A20742E6D2E6B2E206B6579626F617277
:100C400064206669726D7761726520666F722048F4
:100C5000484B42206D6F640A000A092D20566572C8
:100C600073696F6E202D0A000A6D6F7573653A20E7
:100C70006F66660A000A6D6F7573653A206F6E0ABB
:100C8000000A6B6579626F6172643A206F66660A6A
:100C9000000A6B6579626F6172643A206F6E0A00B8
:100CA0000A6D61747269783A206F66660A000A6D8F
:100CB00061747269783A206F6E0A000A6465627521
:100CC000673A206F6E0A000A64656275673A206FA2
:100CD00066660A000A0A626F6F746C6F61646572FF
:100CE0002E2E2E2000433E20000011241FBECFEFE9
:100CF000DAE0DEBFCDBF04B603FE27C080917703E4
:100D000090917803A0917903B0917A038730904B4A
:100D1000A740B04BD1F41092770310927803109251
:100D2000790310927A0314BE84B7877F84BF0FB60D
:100D3000F894A8958091600088618093600010927B
:100D400060000FBEE0E0F8E3099511E0A0E0B1E03B
:100D5000EAE3FBE502C005900D92AA39B107D9F785
:100D600023E0AAE9B1E001C01D92A737B207E1F77D
:100D70000E944B100C949B2D0C9400000FB6809594
:100D80009AE0F8947BE27A95F1F708F0589A08F423
:100D9000589886959A95B1F70FBE08950FB680E8DA
:100DA000F894499BFECF4999FECF96E19A95F1F7C9
:100DB0009CE29A95F1F7869549998068C8F70FBE2D
:100DC00008950FB680E8F89496E19A95F1F79CE2C1
:100DD0009A95F1F7869549998068C8F796E19A95B2
:100DE000F1F7499BFECF0FBE0895FF93EF93E0917B
:100DF0009A01F0919B01309709F00995EF91FF91CD
:100E00000895FC018591803011F0EFDFFBCF08954C
:100E1000FF27E0E230E247FF0CC0419597FF09C091
:100E2000EDE26095709580959095611D711D811D15
:100E3000911D27FF02C0219530E350E2AA27660FDB
:100E4000771F881F991FAA1FA41710F0A41B639572
:100E50005A95A9F7AA3008F0A95FA05DAF93F39562
:100E6000611571058105910541F7ED3211F4EF939C
:100E7000F395F21718F43F93F395FBCF8F91B5DFFD
:100E8000FA95E1F70895E991F9918591803021F083
:100E9000853219F0AADFF9CF089520E0E894559142
:100EA0005532C1F3503311F4689455915A3348F4D4
:100EB000505390F3220F022E220F220F200D250FE8
:100EC000F4CF0EF4219589919991533619F3533744
:100ED00029F1533559F1BC0188279927E8945C36EC
:100EE00021F48991999168945591543639F446EFDB
:100EF0007EF077FF0DC08FEF9FEF0AC055374AE0B5
:100F000039F0583540E121F0523642E009F00895B9
:100F1000FF93EF937DDFEF91FF91B7CFFF93EF93B7
:100F2000FC0181918030B9F360DFFBCFFF93EF9339
:100F300068DFF1CFDF93CF93CDB7DEB72596A3DF80
:100F4000CF91DF91089514B88FEF85B9549A5C98CA
:100F500008958FEF84B980E485B9549A5C9A8FE143
:100F60009EE40197F1F700C0000008958FEF84B967
:100F700080E485B957985F9A87B1806C87B988B14A
:100F8000806C88B92E9A2F980E94A307ECEAF1E0B2
:100F900080E18E0F11928E13FDCFECE9F1E080E13C
:100FA0008E0F11928E13FDCF8CEA91E09093BF01CA
:100FB0008093BE018CE991E09093BD018093BC01C8
:100FC0000895EF92FF920F931F93CF93DF93809139
:100FD000BC019091BD012091BE013091BF013093C1
:100FE000BD012093BC019093BF018093BE015C9B27
:100FF0000E94A907C0E0D0E001E010E080E090E0AE
:10100000FC2FF770EC2FE87025B1207C2F2BAC0162
:1010100033E0440F551F3A95E1F7242B25B928B149
:101020002F73EE2311F0206401C0206828B92AE153
:101030002A95F1F700C0A091BC01B091BD01AC0FA1
:10104000BD1F2C9130E0082E02C0359527950A94DB
:10105000E2F720FD2F9AA5E3AA95F1F70000F6B478
:101060002E98BAE1BA95F1F700C04091BE015091B7
:10107000BF01BA016C0F7D1F4F9B0BC09801082E5A
:1010800001C0220F0A94EAF72095DB013C9123234B
:1010900009C0DB01EC909801082E01C0220F0A94D0
:1010A000EAF72E292C9326B56F2D70E02F1518F036
:1010B00026B530E004C026B530E021503F4F261B56
:1010C000370B2630310558F0A091BC01B091BD011D
:1010D000AC0FBD1F2C91DA01AC0FBD1F2C93BAE1F0
:1010E000BA95F1F700C02F982E9A20EA2A95F1F7C9
:1010F00001968830910509F087CFA091BE01B0918B
:10110000BF01AC0FBD1FE091BC01F091BD01EC0F20
:10111000FD1F9C918081981751F00E94B22460932A
:10112000C0017093C1018093C2019093C3012196C5
:10113000C031D10509F062CF5C9B1BC080916E036A
:10114000853021F080916E03811113C06091C00140
:101150007091C1018091C2019091C3010E94E82465
:10116000613177428105910520F00E94A3070E941A
:10117000332481E0DF91CF911F910F91FF90EF9089
:1011800008952091BE013091BF01F901E80FF11DD2
:10119000808108950C94A9070C94A307569A81FFA7
:1011A00002C05E9A08955E98089588E08093CC000E
:1011B0001092CD00E9ECF0E080818069808380812D
:1011C00088608083EAECF0E080818083EBECF0E0E3
:1011D00080818083559A5D98789408959091C50197
:1011E0002091C4019217D1F030E0F901EA53FE4F8B
:1011F00080812F5F3F4F33272093C401492F50E058
:10120000921718F4241B350B03C0241B350B3395A0
:10121000233031050CF05D9890E008958FEF9FEF3B
:1012200008959091C80095FFFCCF8093CE0008955B
:101230001F920F920FB60F9211242F933F934F934B
:101240005F938F939F93EF93FF938091C50190E0FD
:10125000AC014F5F5F4F2091C401241741F03091E2
:10126000CE00FC01EA53FE4F30834093C50130911C
:10127000C501822F90E0432F50E0841B950B32175D
:1012800008F0939503970CF45D9AFF91EF919F916D
:101290008F915F914F913F912F910F900FBE0F90C3
:1012A0001F9018958091E002089508958091E002C2
:1012B00008950895089508950895CF93DF938D3C80
:1012C0009105B9F1B8F4853B9105A9F148F4833B48
:1012D0009105D1F1843B9105D1F5D0E0C0E23BC04E
:1012E000873B910571F150F18C3C910581F5D0E07F
:1012F000C8E031C08A3E9105C1F040F4823E9105BC
:10130000B1F0893E910519F5D0E124C0813222E087
:10131000920749F0833222E09207D9F08A3891404F
:10132000B1F4D2E017C0D4E015C0D0E213C0D0E4CD
:1013300011C0D0E80FC0D0E0C1E00DC0D0E0C2E0E5
:101340000AC0D0E0C4E007C0D0E0C0E104C0D0E0F3
:1013500001C0D1E0C0E08DEF0E94110983E00E943E
:10136000110983E00E9411098D2F0E9411098C2F11
:10137000DF91CF910C941109CF93DF93EC018DEFA6
:101380000E94110985E00E94110982E00E94110962
:1013900088810E94110989810E9411098A810E9415
:1013A00011098B81DF91CF910C941109CF93DF93B9
:1013B000EC018DEF0E94110989E00E94110981E082
:1013C0000E94110988810E94110980E00E94110980
:1013D0008A810E9411098B810E9411098C810E94CF
:1013E00011098D810E9411098E810E9411098F813E
:1013F000DF91CF910C9411090C94EE08EF92FF92BB
:101400000F931F93CF938C010E94A6247C01C0E010
:10141000C7010E94BE248017910798F40E94EE082D
:101420009C012F3F8FEF380751F02D3041F02A30CB
:1014300041F0EC2FF0E0E853FD4F2083CF5FC73140
:1014400038F3EC2FF0E0E853FD4F108288EC92E087
:10145000CF911F910F91FF90EF9008950C94110977
:1014600081B3881F8827881F0895879A8F9A0895C7
:1014700085B7806885BF85B7806885BF0E94350ABB
:1014800086988E9A81988998559A5D980C94D5087B
:10149000879A8F9808958FB18695817008958FB13E
:1014A00086FB882780F908958093E0020895CF9302
:1014B000DF93FC018491EF012196882321F00E94A3
:1014C0001109FE01F7CFDF91CF910895CF93DF93FC
:1014D000C2EFD1E00E94EE088F3F2FEF920759F044
:1014E0009F938F93DF93CF930E949A070F900F9053
:1014F0000F900F90EFCFDF91CF9108950E94570A80
:101500002FEF89E698E1215080409040E1F700C03C
:10151000000084E690E00E94FE098093C60290934A
:10152000C7029F938F9385EF91E09F938F930E94C3
:101530009A070E94660A0F900F900F900F9080916B
:10154000C6029091C70208950E940D18909315014C
:10155000809314010E94ED1D80E091E00E94081824
:101560000E94480A0E944F0A8111FCCF8DE792E049
:101570000E9401072FEF85EB95E3215080409040BA
:10158000E1F700C0000089E792E00E947E0AEFEFD9
:10159000FBE42DE1E150F0402040E1F700C0000005
:1015A0000E94660A85E792E00E947E0AFC01808123
:1015B000863721F081E792E00C947E0A089588E551
:1015C00092E00E94010782E592E00E947E0A0E945A
:1015D000350A0E94ED1D80911401909115010C9423
:1015E00008180C94870F8F929F92AF92BF92CF9260
:1015F000DF92EF92FF920F931F93CF93DF9392E0CE
:10160000B92E03EA14E029EAE22E24E0F22EAA24FD
:10161000A39433E0932E41E9C42E44E0D42E0E94DB
:10162000FC09EC01019609F441C08091E30281308C
:10163000F9F028F0823009F1833021F134C0CE3F37
:10164000D10519F4A092E302EACFC038D10528F4FD
:10165000DF93CF93FF92EF9204C0DF93CF931F935A
:101660000F930E949A070F900F900F900F90D7CF73
:101670002297C9F4B092E302D2CF2197A1F49092BD
:10168000E302CDCF8091590380FF0AC0DF93CF934F
:10169000DF92CF920E949A070F900F900F900F90B9
:1016A0008C2F0E94540A1092E302B9CF8091E50278
:1016B000811121C08091E40281111DC00E944B0A5A
:1016C00081110AC00E940D188A50914029F00E9491
:1016D000ED1D8AE091E00DC00E944B0A882359F06D
:1016E0000E940D188651914031F00E94ED1D86E157
:1016F00091E00E9408188091E1029091E2020E941C
:10170000BE24893E23E0920708F461C028EE33E04E
:10171000B9010E944B2D629FC001639F900D729F83
:10172000900D11242091E1023091E202820F931F6B
:101730009093E2028093E1020E942510833011F41D
:1017400081E001C080E00E94760F0E94B22428EE62
:1017500033E040E050E00E94732D49015A018CE3D0
:10176000C82ED12CE12CF12CCA01B901A701960198
:101770000E94732D672B682B692B49F50E94EE0F91
:101780002091590320FF23C09F938F931F921F9294
:10179000C501B40120E13EE040E050E00E94732D1D
:1017A000C22FA70196010E94732D3F932F931F9282
:1017B000CF938CE794E09F938F930E949A078DB705
:1017C0009EB70A960FB6F8949EBF0FBE8DBF0E94BB
:1017D0004B0A811107C00E944F0A882319F06E9AA4
:1017E000769802C06E9A769ADF91CF911F910F91F1
:1017F000FF90EF90DF90CF90BF90AF909F908F9031
:1018000008958F929F92AF92BF92CF92DF92EF9204
:10181000FF921F93CF93DF9300D000D0CDB7DEB7F8
:10182000833109F48CC008F05BC08B3009F466C0CA
:101830008C3009F48FC0853009F0FBC10E94B224BE
:1018400028EE33E040E050E00E94732D49015A0138
:101850000E94EE0F9F938F938BEC92E09F938F9358
:101860000E949A07C501B40120E13EE040E050E04B
:101870000E94732D5F934F933F932F9325EC32E09B
:101880003F932F9369837A838B839C830E949A076B
:101890008CE3C82ED12CE12CF12C69817A818B81CB
:1018A0009C81A70196010E94732D5F934F933F93F4
:1018B0002F938FEB92E09F938F930E949A07C5011D
:1018C000B401A70196010E94732D9F938F937F937C
:1018D0006F9389EB92E09F938F930E949A0740C188
:1018E000883361F020F4883109F440C1A2C1873403
:1018F00009F46DC18C3409F456C19BC188E594E0AC
:101900000E94010783E494E00E94010789E294E0C9
:101910000E94010782E094E00E94010787EE93E0B5
:101920000E94010785ED93E00E9401071091E502F6
:1019300011117DC185EB93E00E9401077EC10E94D9
:10194000A40A8DE992E00E947E0A87E992E00E9453
:101950007E0A6BC18CE993E00E9401070E940D187A
:101960008A50914019F08FE291E002C089E291E043
:101970009F938F938EE893E09F938F930E949A0793
:101980008091E4021F928F938FE793E09F938F9350
:101990000E949A070E944B0A0FB6F894DEBF0FBE52
:1019A000CDBF811107C00E944F0A811106C088E394
:1019B00091E005C084E391E002C08BE391E09F9346
:1019C0008F9385E793E09F938F930E949A070E94DD
:1019D000300A1F928F938AE593E09F938F930E9422
:1019E0009A078091E5021F928F9389E493E09F9379
:1019F0008F930E949A0780916E030FB6F894DEBF12
:101A00000FBECDBF8823B9F080916E038130B1F055
:101A100080916E038230A9F080916E038330A1F033
:101A200080916E03843099F080916E03853091F03F
:101A300080E791E011C088E491E00EC080E491E07D
:101A40000BC083E591E008C08BE591E005C085E619
:101A500091E002C082E791E09F938F938AE393E045
:101A60009F938F930E949A0780E393E09F938F93B5
:101A70000E949A070E9425100F900F900F900F90D0
:101A80000F900F90813059F038F0823059F0833048
:101A900061F48AE193E00BC08BE293E008C085E239
:101AA00093E005C08EE193E002C088E193E09F934C
:101AB0008F930E949A070F900F9086E193E09F9377
:101AC0008F930E949A0780916C031F928F938DEFE2
:101AD00092E09F938F930E949A078091D900817022
:101AE0001F928F9383EF92E09F938F930E949A07A8
:101AF0000E94B22428EE33E040E050E00E94732DB3
:101B000069017A019CE3892E912CA12CB12CCA0188
:101B1000B901A50194010E94732D7F936F93C701B2
:101B2000B60120E13EE040E050E00E94732D122F0C
:101B3000A50194010E94732D3F932F931F921F9331
:101B4000C701B60120E831E541E050E00E94732D65
:101B50003F932F9386ED92E09F938F930E949A0775
:101B60000FB6F894DEBF0FBECDBF61C08091E50215
:101B7000811162C01091E402112339F08EEA92E0E3
:101B80000E9401071092E40258C084EA92E00E9489
:101B9000010781E08093E4020E94ED1D86E191E05F
:101BA0000E94081844C00E94300A182F882341F070
:101BB0000E94A40A81E0809369038093E5023DC0FE
:101BC0000E94DF0A109269031092E50230C08091F2
:101BD000E502811102C00E94A40A8BE492E00E94F7
:101BE0007E0A80E492E00E947E0A8CE292E00E94EB
:101BF0007E0A85E292E00E947E0A8BE192E00E94DA
:101C00007E0A84E192E00E947E0A8AE092E00E94CD
:101C10007E0A80E092E00E947E0A8AEF91E00E94B4
:101C20007E0A8091E502811102C00E94DF0A11E064
:101C300004C01091E50201C010E0812F0F900F90B9
:101C40000F900F90DF91CF911F91FF90EF90DF9059
:101C5000CF90BF90AF909F908F900895CF93C82F53
:101C60000E946823827291E009F490E04C2F50E0CA
:101C7000FA013497E934F10508F0D0C0EA5AFF4F71
:101C80000C94952D8BE12DC19111CCC081E629C119
:101C90009111CAC082E625C19111C8C083E621C155
:101CA0009111C6C084E61DC19111C4C085E619C159
:101CB0009111C2C086E615C19111C0C087E611C15D
:101CC0009111BEC088E60DC19111BCC089E609C161
:101CD0009111BAC08AE605C19111B8C08BE601C165
:101CE0009111B6C08CE6FDC09111B4C08DE6F9C06B
:101CF0009111B2C08EE6F5C09111B0C08FE6F1C06F
:101D00009111AEC080E7EDC09111ACC081E7E9C090
:101D10009111AAC082E7E5C09111A8C083E7E1C094
:101D20009111A6C084E7DDC09111A4C085E7D9C098
:101D30009111A2C086E7D5C09111A0C087E7D1C09C
:101D400091119EC088E7CDC091119CC089E7C9C0A0
:101D500091119AC08AE7C5C0911198C081E3C1C0B2
:101D6000911196C082E3BDC0911194C083E3B9C0C4
:101D7000911192C084E3B5C0911190C085E3B1C0C8
:101D800091118EC086E3ADC091118CC087E3A9C0CC
:101D900091118AC088E3A5C0911188C089E3A1C0D0
:101DA000911186C080E39DC088E09BC089E099C006
:101DB00080E297C091117EC08DE293C091117CC0EA
:101DC0008DE38FC091117AC08BE58BC0911178C0E3
:101DD0008DE587C0992309F475C08CE782C09923EB
:101DE00009F472C08CE77DC0911170C08BE379C09B
:101DF00091116EC087E275C091116CC080E671C010
:101E000091116AC08CE26DC0911168C08EE269C008
:101E1000911166C08FE265C080E063C080E261C05E
:101E20008AE05FC081E45DC082E45BC083E459C0A6
:101E300084E457C085E455C086E453C087E451C0AC
:101E400088E44FC089E44DC08AE44BC08BE449C0AC
:101E50008CE447C08DE445C08EE443C08FE441C0AC
:101E600080E53FC081E53DC082E53BC083E539C0E8
:101E700084E537C085E535C086E533C087E531C0E8
:101E800088E52FC089E52DC08AE52BC081E229C0F5
:101E900080E427C083E225C084E223C085E221C01C
:101EA0008EE51FC086E21DC08AE21BC088E219C011
:101EB00089E217C08FE515C08BE213C08BE711C014
:101EC0008DE70FC08CE50DC08CE50BC08AE309C01F
:101ED00082E207C08EE705C08CE303C08EE301C039
:101EE0008FE30E942E0A81E0CF910895833019F488
:101EF000859A7D9A0895813011F4859A06C08230C2
:101F000019F4859A8D9A089585988D98089581E0A1
:101F10000E94760F2FEF81EE94E021508040904098
:101F2000E1F700C0000082E00E94760F2FEF81EE03
:101F300094E0215080409040E1F700C0000081E033
:101F40000E94760F2FEF81EE94E021508040904068
:101F5000E1F700C0000082E00E94760F2FEF81EED3
:101F600094E0215080409040E1F700C0000080E004
:101F70000E94760F80EC80937C0087E080937A004B
:101F800081E980937E0081E080937F008BE38093E2
:101F90007D00849A8C9808958091D90080FF1CC0A0
:101FA00090B331B385988D9AEFE9FFE03197F1F75F
:101FB00000C000008FB185FB882780F920B39072A4
:101FC0002F7D292B20BB91B3232F20729F7D922B35
:101FD00091BB91E08927089580E00895CF93DF9326
:101FE00000D0CDB7DEB7849A8C9A80917A00806851
:101FF00080937A008FE99FE00197F1F700C000001D
:1020000080917A00806480937A0080917A0086FDC6
:10201000FCCF80917800909179009A838983809198
:102020007A008F7780937A00849A8C9829813A81FC
:1020300045E0429FC001439F900D112480559109B6
:102040000F900F90DF91CF9108958091D90080FD7E
:102050000C94CC0F0E94EE0F8C3A2DE0920720F4E6
:1020600081E08093E60205C085379E4010F0109213
:10207000E6028091E602811102C082E0089583E0C9
:102080000895CF93C82F0E94BE068C2F0E94CE10B9
:1020900080E0CF91089584B7877F84BF0FB6F8940E
:1020A000A895809160008861809360001092600024
:1020B0000FBE90E080E80FB6F89480936100909393
:1020C00061000FBE0E9426150E9483158091E200D8
:1020D00084608093E20081E490E10E940424509A9D
:1020E000589A5198599A78948FEF90916E03815035
:1020F000943041F0EFE7FEE33197F1F700C00000C4
:102100008111F3CF8CEC94E00E9401070E94380A01
:102110000E94F10A80EC94E00E9401070E94CE1810
:102120000E944B0A811103C08AE091E002C086E15F
:1021300091E00E94081880EB94E00E9401070E9441
:102140004B0A882319F180916E038530F9F48CEAEB
:1021500094E00E9401070E94CC080E9433240E9450
:1021600033240E9433240E9433240E9433240E948B
:1021700033240E94332480916C03882301F30E944E
:102180005C248823E1F20E947B13D9CF0E94D218ED
:102190000E94F30AD4CF8091F30208959FB7F89478
:1021A0001092EA029FBF90916E03943009F057C0DD
:1021B0009091E9009F703091EC00232F217030FD49
:1021C00020E8922B24E02093E9002091EB0020FFEF
:1021D00043C02091EE0027FF3FC02091E702222359
:1021E00021F02091E80025FF37C01092E70226E099
:1021F0003091E80035FD15C030916E03343061F543
:102200003091EB0035FD28C0215021F481E080930E
:10221000E70222C0EFE9FFE03197F1F700C00000CC
:10222000E7CF8093F1008091E80085FD0AC080919E
:10223000E80080FFFCCF8091E8008E778093E80073
:1022400006C08FB7F89421E02093EA028FBF9F70F9
:102250009093E90080E008959F709093E9008FEFDC
:102260000895CF93DF9300D01F92CDB7DEB79C01C6
:1022700080916E03843019F593E099833B832A8320
:102280009093E9008FEF9091E800815095FD06C092
:1022900095ED9A95F1F700008111F5CF8091E80056
:1022A00085FF0DC040E050E063E070E0CE01019694
:1022B0000E9491138091E8008E778093E8000F9040
:1022C0000F900F90DF91CF910895CF93DF9300D0BF
:1022D0001F92CDB7DEB720916E03243021F522E0A6
:1022E00029839B838A8383E08093E9008FEF909119
:1022F000E800815095FD06C095ED9A95F1F7000034
:102300008111F5CF8091E80085FF0DC040E050E0DD
:1023100063E070E0CE0101960E9491138091E80085
:102320008E778093E8000F900F900F90DF91CF9100
:10233000089520916E032430F1F422E02093E90007
:102340002FEF3091E800215035FD06C035ED3A956C
:10235000F1F700002111F5CF2091E80025FF0BC017
:1023600040E050E065E070E00E9491138091E80049
:102370008E778093E8000895CF93DF9320916E03CA
:10238000243039F521E02093E9002FEF3091E80067
:10239000215035FD06C035ED3A95F1F700002111C9
:1023A000F5CF2091E80025FF14C0EC0140E050E09B
:1023B00068E070E00E9491138091E8008E7780932E
:1023C000E80088E0FE01ABEEB2E001900D928A9544
:1023D000E1F7DF91CF9108958BED94E00E94010722
:1023E00080916D03811109C00E9426150E948315FA
:1023F0008091E20084608093E200089587ED94E08C
:102400000E94010710926D03089508952091E8023B
:102410002F5F822F62E30E943F2D992319F02093B2
:10242000E80208951092E8028091EA02882371F18F
:1024300080916E03843041F58091E9008F70209186
:10244000EC00922F917020FD90E8892B94E09093FE
:10245000E9009091EB0090FF14C09091EE0097FF7F
:1024600010C09091E80095FF03C01092F100F9CFE1
:102470009091E80090FF05C09091E8009E779093BE
:10248000E8008F708093E9001092EA02089542E01C
:1024900061EC81E00E94A01442E061EC82E00E94C5
:1024A000A01442E061EC83E00E94A01442E261ECDF
:1024B00084E00C94A01480917003833009F453C01D
:1024C00030F4813071F0823009F48CC008958A3084
:1024D00009F478C08B3009F45EC0893009F09AC0E5
:1024E00020C080916F03813A09F094C08091E80088
:1024F000877F8093E8008091730390917403892B08
:1025000021F468E08BEE92E003C060E080E090E0B0
:1025100070E00E94DC138091E8008B778093E800E4
:10252000089580916F03813209F074C08091730324
:1025300090917403892B09F06DC08091E800877F2A
:102540008093E8008091E80082FD05C080916E03D1
:102550008111F8CF5FC08091F1008093F3028091E8
:10256000E8008B7753C080916F03813A09F052C025
:102570008091730390917403892B09F04BC0809173
:10258000E800877F8093E8008091E80080FFFCCF1F
:102590008091200136C080916F038132D9F58091FE
:1025A000730390917403892BA9F58091E800877FCC
:1025B0008093E8000E94D5148091710380932001DC
:1025C0000C94ED1D80916F03813221F58091E8001C
:1025D000877F8093E8000E94D514809172038093D6
:1025E000F402089580916F03813AA1F48091E8008C
:1025F000877F8093E8008091E80080FFFCCF809186
:10260000F4028093F1008091E8008E778093E800D7
:102610000C94D51408958091F3028093E9021092EE
:10262000F30280E00E94CE080E9491190C94ED1DE7
:102630000C940B130E9470248091E9028093F302A2
:1026400008950C941A13292F332723303105C9F02C
:1026500064F42130310581F02230310509F043C0A6
:1026600084E790E027E035E042C021323105F1F007
:102670002232310541F137C082E190E02BE735E0AD
:1026800036C099278130910541F08230910541F0A3
:10269000892B49F5E3E0F5E005C0E3EFF4E002C083
:1026A000EFEDF4E0849190E09F0121C06430D8F414
:1026B000E62FF0E0EE0FFF1FE857FE4F208131813B
:1026C00089E090E014C0643070F470E0FB01EE0F1C
:1026D000FF1FE058FE4F20813181FB01E458FE4F7F
:1026E000808190E004C080E090E020E030E0FA01DA
:1026F00031832083089580E189BD82E189BD09B4D9
:1027000000FEFDCF8091D8008F7D8093D80080910E
:10271000E00082608093E0008091E00081FDFCCFCA
:102720000895CF92DF92EF92FF920F931F93CF9372
:10273000DF93EC018B016A010E94F414811133C014
:10274000C114D10439F0F60180819181081B190B65
:10275000C80FD91FE12CF12C0115110519F1809139
:10276000E80085FD16C08091E8008E778093E80030
:10277000C114D10449F0F60180819181E80EF91E5F
:10278000F182E08285E00FC00E94F414882321F3D7
:102790000AC089918093F10001501109FFEFEF1AEF
:1027A000FF0ADACF80E0DF91CF911F910F91FF9068
:1027B000EF90DF90CF9008952091750330917603CC
:1027C0002617370748F06115710539F42091E800A4
:1027D0002E772093E80001C0B90140E06115710532
:1027E000A9F120916E03222309F443C0253009F496
:1027F00042C02091E80023FD40C02091E80022FD66
:1028000032C02091E80020FFE9CF4091F3002091F1
:10281000F20030E0342BFC01CF016115710559F055
:102820002830310540F481918093F10061507109A5
:102830002F5F3F4FF1CF41E02830310509F040E0F4
:102840002091E8002E772093E800C8CF4111C9CF2E
:102850000AC080916E03882361F0853061F0809119
:10286000E80083FD0AC08091E80082FFF2CF80E09B
:10287000089582E0089583E0089581E0089520910D
:102880007503309176032617370748F061157105F7
:1028900039F42091E8002E772093E80001C0B901B7
:1028A000FC0120E06115710591F180916E03882390
:1028B00009F440C0853009F43FC08091E80083FDF1
:1028C0003DC08091E80082FD2FC08091E80080FF2C
:1028D000E9CF2091F3008091F20090E0922B6115F6
:1028E000710559F08830910540F424912093F1004E
:1028F0003196615071090196F2CF21E0089709F0F5
:1029000020E08091E8008E778093E800CBCF211102
:10291000CCCF0AC080916E03882361F0853061F0CE
:102920008091E80083FD0AC08091E80082FFF2CF29
:1029300080E0089582E0089583E0089581E008959D
:10294000982F973058F59093E900981739F07091C7
:10295000EC002091ED005091F00003C0242F762F61
:1029600050E021FF19C03091EB003E7F3093EB0027
:102970003091ED003D7F3093ED003091EB00316000
:102980003093EB007093EC002093ED005093F00037
:102990002091EE0027FF07C09F5FD3CF8F708093F9
:1029A000E90081E0089580E0089580916F0387FF3A
:1029B00011C08091E80082FD05C080916E038111F5
:1029C000F8CF11C08091E8008B770BC080916E0327
:1029D000882349F08091E80080FFF8CF8091E800DB
:1029E0008E778093E80008952091E4003091E5000F
:1029F00095E64091EC00842F817040FF22C08091C9
:102A0000E80080FD1CC080916E03882391F0853022
:102A100091F08091EB0085FD10C04091E400509151
:102A2000E5004217530729F39A01915011F784E00A
:102A3000089582E0089583E0089581E0089580E09C
:102A400008954091E80042FFDECF08950E9494155A
:102A50000E949C15E0EEF0E0808181608083E8EDCB
:102A6000F0E080818F77808319BCA7EDB0E08C9176
:102A70008E7F8C9380818F7E808310926D0308956A
:102A80000F931F93CF93DF930E9494150E949C1580
:102A9000C8EDD0E088818F778883888180688883BB
:102AA00088818F7D888319BC10926E0310926A030F
:102AB00010926C0310926B0300EE10E0F80180811D
:102AC0008B7F808388818160888342E060E080E042
:102AD0000E94A014E1EEF0E080818E7F8083E2EE20
:102AE000F0E0808181608083808188608083F8014C
:102AF00080818E7F8083888180618883DF91CF9100
:102B00001F910F910895E8EDF0E080818F7E808322
:102B1000E7EDF0E080818160808384E082BF81E026
:102B200080936D030C944015E8EDF0E080818E7F7A
:102B300080831092E20008951092DA001092E10072
:102B400008951F920F920FB60F9211242F933F9367
:102B50004F935F936F937F938F939F93AF93BF93A5
:102B6000EF93FF938091E10082FF0BC08091E20020
:102B700082FF07C08091E1008B7F8093E1000E947B
:102B800006128091DA0080FF1FC08091D80080FF7C
:102B90001BC08091DA008E7F8093DA008091D9008B
:102BA00080FF0DC080E189BD82E189BD09B400FECE
:102BB000FDCF81E080936E030E94EC1105C019BC2B
:102BC00010926E030E94FE118091E10080FF19C0F7
:102BD0008091E20080FF15C08091E2008E7F80939B
:102BE000E2008091E20080618093E2008091D80051
:102BF00080628093D80019BC85E080936E030E94A8
:102C000018138091E10084FF30C08091E20084FFBE
:102C10002CC080E189BD82E189BD09B400FEFDCFF1
:102C20008091D8008F7D8093D8008091E1008F7EC5
:102C30008093E1008091E2008F7E8093E20080919A
:102C4000E20081608093E20080916A03882311F0A2
:102C500084E007C08091E30087FD02C081E001C0ED
:102C600083E080936E030E9421138091E10083FF33
:102C700029C08091E20083FF25C08091E100877F19
:102C80008093E10082E080936E0310926A0380914A
:102C9000E1008E7F8093E1008091E2008E7F80933F
:102CA000E2008091E20080618093E20042E060E017
:102CB00080E00E94A0148091F00088608093F00072
:102CC0000E940512FF91EF91BF91AF919F918F915B
:102CD0007F916F915F914F913F912F910F900FBE18
:102CE0000F901F9018951F920F920FB60F921124FC
:102CF0002F933F934F935F936F937F938F939F9304
:102D0000AF93BF93CF93DF93EF93FF93C091E9000D
:102D1000CF708091EC00D82FD17080FDD0E8109258
:102D2000E9008091F000877F8093F00078940E9402
:102D3000B7161092E9008091F00088608093F0004F
:102D4000CD2BCF70C093E900FF91EF91DF91CF9130
:102D5000BF91AF919F918F917F916F915F914F91B3
:102D60003F912F910F900FBE0F901F9018951F93BA
:102D7000CF93DF93CDB7DEB7AA970FB6F894DEBF37
:102D80000FBECDBFEFE6F3E088E08E0F9091F1002B
:102D900091938E13FBCF0E945B128091E80083FF1A
:102DA0001FC180916F0390917003492F50E04A300A
:102DB000510508F015C1FA01E156FF4F0C94952D0D
:102DC000803881F0823809F00BC1809173038F70D5
:102DD0008093E9008091EB0085FB882780F91092B1
:102DE000E90006C080916B0390916C0391118260A1
:102DF0009091E800977F9093E8008093F100109203
:102E0000F100C8C0282F2D7F09F0EAC0882319F0EF
:102E1000823061F0E5C080917103813009F0E0C03B
:102E2000933009F080E080936C032BC08091710394
:102E3000811127C0809173038F7009F4D1C08093F2
:102E4000E9002091EB0020FF1CC0933021F4809119
:102E5000EB00806214C09091EB0090619093EB00C6
:102E600021E030E0A90102C0440F551F8A95E2F726
:102E70004093EA001092EA008091EB008860809312
:102E8000EB001092E9008091E800877F86C08111F5
:102E9000A7C0109171031F778091E3008078812B88
:102EA0008093E3008091E800877F8093E8000E9490
:102EB000D5148091E80080FFFCCF8091E30080680A
:102EC0008093E300111102C082E001C083E080938F
:102ED0006E0386C08058823008F082C080917103F2
:102EE000909172038C3D53E0950779F583E08A83D6
:102EF0008AE289834FB7F894DE01139620E03EE022
:102F000051E2E32FF0E050935700E49120FF03C01B
:102F1000E295EF703F5FEF708E2F90E0EA3010F097
:102F2000C79601C0C0968D939D932F5F243149F7BA
:102F30004FBF8091E800877F8093E8006AE270E0ED
:102F4000CE0101960E94DC1314C0AE014F5F5F4FAB
:102F5000609173030E942313BC01892B09F440C0C4
:102F60009091E800977F9093E80089819A810E9470
:102F70003F148091E8008B778093E80031C080385F
:102F800079F58091E800877F8093E80080916A035B
:102F90008093F1008091E8008E778093E8000E9492
:102FA000D5141EC081111CC0909171039230C0F4E1
:102FB0008091E800877F8093E80090936A030E94E5
:102FC000D51480916A03811106C08091E30087FDCA
:102FD00002C081E001C084E080936E030E9447122A
:102FE0008091E80083FF0AC08091E800877F80938A
:102FF000E8008091EB0080628093EB00AA960FB608
:10300000F894DEBF0FBECDBFDF91CF911F91089521
:103010009093FA028093F90208958091F9029091B9
:10302000FA020895E091F902F091FA02309721F046
:103030000190F081E02D099480E00895EF92FF92D5
:103040000F931F93CF93DF93E091F902F091FA026F
:103050003097B1F18C010280F381E02D09958091C8
:10306000590382FF2DC080FF04C088E996E00E94CA
:103070000107E80118E082E9E82E86E0F82E809149
:10308000590380FF0BC088811F928F93FF92EF92AC
:103090000E949A070F900F900F900F901150219659
:1030A0001111EDCF8091590380FF0AC080E996E0AD
:1030B000DF91CF911F910F91FF90EF900C9401073A
:1030C000DF91CF911F910F91FF90EF900895E091C4
:1030D000F902F091FA02309721F00480F581E02D99
:1030E00009940895CF93DF93EC018091F7029091BA
:1030F000F802C817D90709F1D093F802C093F70274
:10310000E091F902F091FA023097B9F00680F78168
:10311000E02DCE0109958091590382FF0EC080FFFA
:103120000CC0DF93CF9382E896E09F938F930E9429
:103130009A070F900F900F900F90DF91CF91089505
:10314000CF93DF93EC018091F5029091F602C817BE
:10315000D90709F1D093F602C093F502E091F90284
:10316000F091FA023097B9F00084F185E02DCE019C
:1031700009958091590382FF0EC080FF0CC0DF9338
:10318000CF9382E796E09F938F930E949A070F90C8
:103190000F900F900F90DF91CF9108950E949D2482
:1031A0000C94B607CF92DF92EF92FF920F931F938A
:1031B000CF93DF9300D000D000D0CDB7DEB70E9410
:1031C000E1078CEFC82E82E0D82E00E010E0E02E60
:1031D000802F0E94C108F60141916F01F42EF8265C
:1031E000B1F40F5F1F4F0031110589F78FEF89830D
:1031F0008A831B820E94A6248160782F9D838C8302
:1032000049815A816B818D810E94C61947C0909176
:10321000590391FF04C08E830E9492198E8120E091
:1032200030E04F2D50E0922FBA01022E02C075956A
:1032300067950A94E2F760FF2BC02983EA8221E0B8
:1032400030E0690102C0CC0CDD1C9A95E2F790E0F9
:103250008C219D21892B09F420E02B830E94A62438
:103260008160782F9D838C8349815A816B818D8108
:103270000E94C61949815A816B817C818D810E948F
:103280002024F801E450FD4F8081C826C08206C08A
:103290002F5F3F4F2830310531F6A3CF0E941F2406
:1032A0000E9493271091FB020E941218181741F1F7
:1032B0000E9412188093FB029091590392FF0EC056
:1032C00090FF0CC01F928F9383EA96E09F938F9399
:1032D0000E949A070F900F900F900F908091FB0221
:1032E00026960FB6F894DEBF0FBECDBFDF91CF910B
:1032F0001F910F91FF90EF90DF90CF900C943124AD
:1033000026960FB6F894DEBF0FBECDBFDF91CF91EA
:103310001F910F91FF90EF90DF90CF9008950C9444
:10332000CE080895EF92FF920F931F93CF93DF93F0
:103330008CEB96E00E940107C0E0D0E08EE2E82E20
:1033400081E0F82E0EEA16E08C2F0E94C1080E9440
:103350000924FF92EF921F928F93DF93CF931F93D5
:103360000F930E949A0721968DB79EB708960FB6C5
:10337000F8949EBF0FBE8DBFC031D10529F7DF91F4
:10338000CF911F910F91FF90EF900895CF93DF930E
:10339000CDB7DEB72B970FB6F894DEBF0FBECDBF0B
:1033A000942F4F83252F588769877A878B874A8583
:1033B0005B85452B21F02F3F09F59F3FF9F4DE0196
:1033C000119686E0FD0111928A95E9F785E0FE01EC
:1033D000379601900D928A95E1F749815A816B8168
:1033E0007C818D819E810E94A1202B960FB6F8943E
:1033F000DEBF0FBECDBFDF91CF9108954F815885BD
:1034000069857A858B850E942024D9CFCF93882324
:1034100009F465C0C82F8CEF8C0F813A20F080E54D
:103420008C0F8E3248F48C2F0E94B92A811157C01C
:103430008C2F0E942C230CC080E28C0F883058F413
:10344000C77081E001C0880FCA95EAF70E946B231C
:10345000CF910C94AF238BE58C0F833078F4C53A71
:1034600029F0C63A31F083E890E005C081E890E0A9
:1034700002C082E890E0CF910C94721888E58C0F1E
:10348000853168F5C83A89F0C93A91F0CA3A99F09D
:10349000CB3AA1F0CC3AA9F0CD3AB1F0CE3AB9F09E
:1034A000CF3AC1F080E090E017C082EE90E014C007
:1034B00089EE90E011C08AEE90E00EC085EB90E0BE
:1034C0000BC086EB90E008C083EB90E005C084EB76
:1034D00090E002C087EB90E0CF910C94A018CF91C0
:1034E0000895882349F19CEF980F913A20F090E5D8
:1034F000980F9E3218F40E9449230DC090E2980F55
:10350000983058F4877091E001C0990F8A95EAF7D6
:10351000892F0E9471230C94AF239BE5980F933061
:1035200020F480E090E00C947218885A853120F4E1
:1035300080E090E00C94A0180895882321F00E9468
:103540006B230C94AF230895882321F00E947123EC
:103550000C94AF230895BF92CF92DF92EF92FF9227
:103560000F931F93CF93DF9300D000D000D0CDB73F
:10357000DEB725E0FC01DE01119601900D922A953F
:10358000E1F7FC0140813181F280258122952F7085
:1035900063817481672B09F4FEC23F3F19F44F3FEA
:1035A00009F4F9C26C0149833A8389819A812E8397
:1035B0000E94EB22182FB92E0E94EA220E94FA21C3
:1035C000EB2DE295EF70F0E0E755FF4F2E810C9464
:1035D000952D8B2D807F9B2D9F70092F882311F0B7
:1035E0000295007FFF2049F0002309F481C2802F5B
:1035F0000E947E230E94AF237BC2812F0E94711AFA
:10360000002309F4C8C2802F0E94842326960FB697
:10361000F894DEBF0FBECDBFDF91CF911F910F9108
:10362000FF90EF90DF90CF90BF900C94AF238B2D45
:10363000807F9B2D9F70092F803211F00295007FB3
:10364000112319F0113009F12AC0FF20B1F0802FA9
:10365000222351F1213041F526960FB6F894DEBFB2
:103660000FBECDBFDF91CF911F910F91FF90EF90D3
:10367000DF90CF90BF900C948E23222319F021303D
:1036800009F489C20E9497232DC0FF20F1F0263053
:1036900008F081C20E946823802329F023C0FF2004
:1036A000F9F0211116C0802F26960FB6F894DEBFD0
:1036B0000FBECDBFDF91CF911F910F91FF90EF9083
:1036C000DF90CF90BF900C949D1A253008F063C214
:1036D00009C0F601858180FF0BC28F708583E3CF1F
:1036E00021111BC2802F82C12B2D26952695237078
:1036F00030E02115310521F021303105D1F04BC2E8
:10370000FF2021F0812F9B2D937002C080E090E07C
:1037100026960FB6F894DEBF0FBECDBFDF91CF91D6
:103720001F910F91FF90EF90DF90CF90BF900C947E
:103730007218FF2021F0812F9B2D937002C080E032
:1037400090E026960FB6F894DEBF0FBECDBFDF9196
:10375000CF911F910F91FF90EF90DF90CF90BF908E
:103760000C94A018812FFF2019F00E94192602C086
:103770000E94812626960FB6F894DEBF0FBECDBFFD
:10378000DF91CF911F910F91FF90EF90DF90CF903D
:10379000BF900C9406278B2D837009F07BC0F1102D
:1037A000FAC1812F829586958770880F880F912F97
:1037B0009F70C92ED12CE12CF12C082E04C0CC0C0A
:1037C000DD1CEE1CFF1C0A94D2F714FF12C04FE060
:1037D00050E060E070E004C0440F551F661F771F83
:1037E0008A95D2F7CB01BA01609570958095909536
:1037F00003C060E070E0CB012B2D26952695237049
:10380000422F50E042305105D9F04330510569F163
:103810006C297D298E299F294130510551F1269629
:103820000FB6F894DEBF0FBECDBFDF91CF911F91D1
:103830000F91FF90EF90DF90CF90BF900C940F22EC
:103840006C297D298E299F2926960FB6F894DEBF14
:103850000FBECDBFDF91CF911F910F91FF90EF90E1
:10386000DF90CF90BF900C9421220E940F22C701BD
:10387000B60126960FB6F894DEBF0FBECDBFDF911E
:10388000CF911F910F91FF90EF90DF90CF90BF905D
:103890000C94FD21FF2019F08B2D817001C08695BD
:1038A000882309F478C1812F829586958770880FC7
:1038B000880F912F9F70C92ED12CE12CF12C082E4E
:1038C00004C0CC0CDD1CEE1CFF1C0A94D2F714FFC4
:1038D00012C04FE050E060E070E004C0440F551F9C
:1038E000661F771F8A95D2F7CB01BA016095709554
:1038F0008095909503C060E070E0CB012B2D26955C
:1039000026952370422F50E042305105D9F04330C4
:10391000510569F16C297D298E299F294130510576
:1039200051F126960FB6F894DEBF0FBECDBFDF91E2
:10393000CF911F910F91FF90EF90DF90CF90BF90AC
:103940000C94C6226C297D298E299F2926960FB6B4
:10395000F894DEBF0FBECDBFDF91CF911F910F91C5
:10396000FF90EF90DF90CF90BF900C94D8220E94F0
:10397000C622C701B60126960FB6F894DEBF0FBE69
:10398000CDBFDF91CF911F910F91FF90EF90DF900E
:10399000CF90BF900C94B422103FC9F128F480E47A
:1039A000810F803250F09FC0123F09F461C008F4CB
:1039B0004AC0133F09F471C096C0012F00718B2DCE
:1039C0008F71FF2051F00E944D22812F002319F0AA
:1039D0008295807F69CE8F7067CE0E946E22812F84
:1039E000002319F08295807F01C08F7026960FB654
:1039F000F894DEBF0FBECDBFDF91CF911F910F9125
:103A0000FF90EF90DF90CF90BF900C94A41AFF200E
:103A1000B1F0253008F0BFC08B2D8F7126960FB600
:103A2000F894DEBF0FBECDBFDF91CF911F910F91F4
:103A3000FF90EF90DF90CF90BF900C9493222630B0
:103A400008F0A9C0E9CFFF20A9F08B2D8F71269631
:103A50000FB6F894DEBF0FBECDBFDF91CF911F919F
:103A60000F91FF90EF90DF90CF90BF900C944D227C
:103A7000FF2059F38B2D8F7126960FB6F894DEBF79
:103A80000FBECDBFDF91CF911F910F91FF90EF90AF
:103A9000DF90CF90BF900C946E22FF2099F08B2D79
:103AA0008F7126960FB6F894DEBF0FBECDBFDF91A3
:103AB000CF911F910F91FF90EF90DF90CF90BF902B
:103AC0000C94382226960FB6F894DEBF0FBECDBFF9
:103AD000DF91CF911F910F91FF90EF90DF90CF90EA
:103AE000BF900C943322FF20A9F0222309F4ADCF1C
:103AF000812F26960FB6F894DEBF0FBECDBFDF91A3
:103B0000CF911F910F91FF90EF90DF90CF90BF90DA
:103B10000C94061A222309F4ADCF812F26960FB6F6
:103B2000F894DEBF0FBECDBFDF91CF911F910F91F3
:103B3000FF90EF90DF90CF90BF900C94711A4B2DB7
:103B40004F70612FC6010E94932526960FB6F894F8
:103B5000DEBF0FBECDBFDF91CF911F910F91FF90C0
:103B6000EF90DF90CF90BF900C9445214B2D4F707C
:103B7000612FC60126960FB6F894DEBF0FBECDBFEB
:103B8000DF91CF911F910F91FF90EF90DF90CF9039
:103B9000BF900C94962526960FB6F894DEBF0FBE04
:103BA000CDBFDF91CF911F910F91FF90EF90DF90EC
:103BB000CF90BF9008950E948B230E945A230E94A9
:103BC000AF230E9438280E94062780E090E00E94E0
:103BD000721880E090E00C94A0180E947B230C9453
:103BE000DB1D0E94EB22292F22952F7030E02C3014
:103BF00031054CF42A303105C4F422503109223009
:103C0000310540F023C02C303105D1F02F30310583
:103C1000B9F01CC0853A28F48430B0F4823028F41E
:103C200013C090E2980F983078F0883E30F4803ED0
:103C300058F48450813A50F407C0803F39F404C0EE
:103C400093FB882780F9089581E0089580E0089526
:103C5000CF93DF9300D000D01F92CDB7DEB70F9087
:103C60000F900F900F900F90DF91CF910895CF9309
:103C7000DF9300D000D000D0CDB7DEB726960FB6C8
:103C8000F894DEBF0FBECDBFDF91CF9108951F9393
:103C9000CF93DF93C0910C0316E080910D03C817FA
:103CA00099F0D0E01C9FF0011D9FF00D1124E25F00
:103CB000FC4F4081518162817381848195810E9492
:103CC000371E2196C770E9CFDF91CF911F910895DC
:103CD00040913E0350913F03609140037091410336
:103CE00080914203909143030C94371E80914303CB
:103CF00082958F7009F054C080914003882309F4A5
:103D00004FC080910C03A0910D0360913E03709110
:103D10003F034091410350914203B6E08A1709F4F2
:103D20003FC090E041155105C1F17F3F11F46F3F55
:103D3000A1F1B89FF001B99FF00D1124E25FFC4F93
:103D4000218172132AC02081621327C02281211190
:103D500024C0238134812417350710F42150310900
:103D6000241B350B2C323140C0F4209143032F70BB
:103D700020612093430326E0289FF001299FF00D46
:103D80001124ED5EFC4F80818F70806180838EE313
:103D900093E00E94AB1A0C94471E01968770BECF29
:103DA0000895CF92DF92EF92FF920F931F93CF93DC
:103DB000DF93CDB7DEB762970FB6F894DEBF0FBEC4
:103DC000CDBF8C0185E0F801DE011D9601900D92BA
:103DD0008A95E1F7D8014C9111965C911197129652
:103DE0006C9112971396CD90DC90149730913E030E
:103DF00070913F038091410390914203009709F431
:103E000073C17F3F19F43F3F09F46EC1E090400356
:103E1000EE2009F4C5C020914303C816D90650F01E
:103E2000F601E81BF90BCF01FF24F3948C3291408B
:103E3000C8F009C0809590958C0D9D1DFF24F394CA
:103E40008C32914078F0F12C207F09F0C6C07C2D97
:103E5000D98AC88A89890E94281E8EE393E00E942D
:103E6000AB1AB1C0822F807F09F045C0751313C013
:103E7000341311C061110FC02F70206120934303D0
:103E80000E94681E8EE393E00E94AB1A8091430368
:103E9000F80185832EC0CD2819F15F3F11F44F3F03
:103EA000F9F0F62E61111CC080910C0320910D03D6
:103EB00036E0821709F45BC090E0389FF001399F2B
:103EC000F00D1124E25FFC4F7181571306C0708121
:103ED000471303C07281711103C001968770E9CF47
:103EE000F62E662309F41DC18091430381608093FF
:103EF0004303F12C16C1751309C0341307C06111B7
:103F000005C080914303F8018583C8C04D875E8753
:103F10008D859E856A8B0E94F11D6A898823E1F157
:103F20006623D1F120914303822F82958F7090E018
:103F3000029774F080913E0390913F0398878F839E
:103F40001986DB86CA862C87CE0107960E94AB1A9B
:103F500086E0F801AEE3B3E001900D928A95E1F7B7
:103F60000E94761E0E94681EFF24F394DAC04D87DB
:103F70005E878D859E850E94EB22292F22952F70CA
:103F800030E0223031050CF0BFC09F7009F0B9C09D
:103F9000805E883008F4C5C0C8010E94AB1AE4CF27
:103FA000C816D90608F453C0F601E81BF90BCF0177
:103FB0008C32914008F453C0F12C7C2DD98AC88AE8
:103FC00089890E94281EEEE3F3E086E0DF011D925E
:103FD0008A95E9F70E94681EA4C0751314C03413B3
:103FE00012C0611110C080914303F8018583C8019C
:103FF0000E94AB1A86E0EEE3F3E0DF011D928A95A2
:10400000E9F7FE2C8EC04D875E878D859E856A8B75
:104010000E94F11D6A89882309F4BECF662309F442
:10402000BBCF20914303822F82958F7090E002973F
:104030000CF48ECF80913E0390913F039A83898345
:104040001B82DD82CC822E83CE0101967FCF8095AC
:1040500090958C0D9D1D8C32914008F0ADCFF62EC1
:10406000662309F499CF75132EC034132CC0209108
:10407000430320FD1FC0822F82958F70D9F0D80195
:1040800015962C9315978F3049F08F5F982F929546
:10409000907F822F8F70892B15968C93C8010E9478
:1040A000AB1A86E0F801AEE3B3E001900D928A9579
:1040B000E1F790CF86E0F801AEE3B3E001900D9216
:1040C0008A95E1F72EC04D875E878D859E850E947B
:1040D000F11D81113DCF80914303816080934303A3
:1040E000C8010E94AB1A1DC0662309F455CF4D8745
:1040F0005E878D859E850E94F11D882309F44CCF33
:1041000027CF811145CF0DC0243031050CF044CFAD
:104110009F7009F43DCFD80115969C91907F09F0CE
:1041200037CF8F2D62960FB6F894DEBF0FBECDBF8E
:10413000DF91CF911F910F91FF90EF90DF90CF9083
:1041400008951F93CF93DF93CDB7DEB72C970FB6AB
:10415000F894DEBF0FBECDBF4F83588769877A873B
:104160008B879C87CE0107960E94D11E882369F019
:104170008F8198852A853B85232BF1F19F3F09F09C
:1041800063C08F3F09F060C037C086E0FE013796FC
:10419000DE01119601900D928A95E1F76F81788585
:1041A000EA85FB85309741F17F3F11F46F3F21F1A4
:1041B00020910D0330E0C901019687709927409145
:1041C0000C0350E08417950709F447C069837A838C
:1041D000FD83EC8396E0929FD001939FB00D112454
:1041E000A25FBC4FFE01319601900D929A95E1F7C6
:1041F00080930D030E94471E16E080910C0390915E
:104200000D038917C1F1189FC0011124825F9C4FD3
:104210000E94D11E882379F1E0910C031E9FF001CA
:104220001124E25FFC4F408151816281738184815E
:1042300095810E94371E80910C0390E00196877053
:10424000992780930C03D9CF4F81588569857A854A
:104250008B859C850E94371ECFCF0E94ED1D10924A
:104260000D0310920C03EEE3F3E086E0DF011D92F4
:104270008A95E9F7C1CF2C960FB6F894DEBF0FBE32
:10428000CDBFDF91CF911F910895DF92EF92FF9202
:104290000F931F93CF93DF93FC01892B09F48AC0FE
:1042A000E12CF12CDD24D394EF0121968491853704
:1042B00009F461C058F4843708F04EC0843008F027
:1042C0006AC08130D1F0823071F174C0883709F44E
:1042D0005DC050F4863709F455C0873709F06AC0CD
:1042E0008E2D0E94782354C09CE7980F903708F0D9
:1042F00061C08F770E94711A50C08F010E5F1F4FEF
:10430000FE01849190E2980F983050F48770FD2D53
:1043100001C0FF0F8A95EAF78F2F0E947E2314C0F9
:104320000E94061A13C08F010E5F1F4FFE01C49139
:1043300080E28C0F883060F4C7708D2D01C0880F2B
:10434000CA95EAF70E9484230E94AF23E80125C0A2
:104350008C2F0E94711AFACF9F012E5F3F4FFE01F2
:10436000C491CC2369F08FE99FE00197F1F700C079
:104370000000C150F6CF9F012E5F3F4FFE01F49029
:10438000E9010BC00E946823E82E07C00E947B232E
:104390000E94AF2302C00E94061A8F2D882341F08D
:1043A000EFE9FFE03197F1F700C000008150F6CF50
:1043B000FE017ACFDF91CF911F910F91FF90EF9087
:1043C000DF900895609348037093490380934A03F4
:1043D00090934B030E942F240C94DB1D60934403A5
:1043E0007093450380934603909347030E943024C3
:1043F0000C94DB1D08950C94E2210F931F93009100
:1044000048031091490320914A0330914B03602BDC
:10441000712B822B932B1F910F910C94E2210F9300
:104420001F93009148031091490320914A03309152
:104430004B0360237123822393231F910F910C94CC
:10444000E2210F931F93009148031091490320919B
:104450004A0330914B0360277127822793271F91CE
:104460000F910C94E22160E070E0CB010C94EE21FE
:104470000F931F9341E050E060E070E08A019B01E0
:1044800004C0000F111F221F331F8A95D2F7C901E4
:10449000B8011F910F910C94EE210F931F9341E0EF
:1044A00050E060E070E004C0440F551F661F771FA6
:1044B0008A95D2F78091440390914503A0914603D9
:1044C000B09147038A019B01082B192B2A2B3B2B08
:1044D000C901B8011F910F910C94EE210F931F9306
:1044E00041E050E060E070E004C0440F551F661FDB
:1044F000771F8A95D2F74095509560957095809179
:10450000440390914503A0914603B09147038A016B
:104510009B01082319232A233B23C901B8011F91BA
:104520000F910C94EE210F931F9341E050E060E057
:1045300070E004C0440F551F661F771F8A95D2F79D
:104540008091440390914503A0914603B0914703A5
:104550008A019B01082719272A273B27C901B8018F
:104560001F910F910C94EE210F931F930091440320
:10457000109145032091460330914703602B712B26
:10458000822B932B1F910F910C94EE210F931F936D
:104590000091440310914503209146033091470355
:1045A00060237123822393231F910F910C94EE219A
:1045B0000F931F93009144031091450320914603EC
:1045C0003091470360277127822793271F910F910E
:1045D0000C94EE210895CF92DF92EF92FF920F9309
:1045E0001F93CF93DF938C01C0904803D090490371
:1045F000E0904A03F0904B034091440350914503EF
:104600006091460370914703C42AD52AE62AF72A07
:10461000CFE1D0E0D701C6010C2E04C0B695A79516
:10462000979587950A94D2F780FF07C0B8018C2F21
:104630000E9469258130910531F4219758F7B8011E
:1046400080E00E946925DF91CF911F910F91FF902B
:10465000EF90DF90CF9008952091210130912201B9
:10466000F90132969FEF40E05191581789F09F3F32
:1046700019F4511101C0942F4F5F4630A9F79F3FA5
:1046800039F0F901E90FF11D97FDFA95828308953C
:1046900008952091210130912201F9013296285F7D
:1046A0003F4F9081981301C010823196E217F307B3
:1046B000C1F7089581E090E0E0912101F09122019D
:1046C000E80FF91F1082019688309105A9F7089527
:1046D00080915803089590915803892B8093580333
:1046E00008958095909158038923809358030895E5
:1046F000809358030895109258030895909157039A
:10470000892B8093570308958095909157038923AF
:1047100080935703089510925703089580934E0392
:104720000E94A62490934D0380934C030895109209
:104730004E0310924D0310924C0308958091210175
:1047400090912201FC0131969C01285F3F4F80E04F
:10475000919191118F5FE217F307D1F70895E091DE
:104760002101F0912201809158038083E091210181
:10477000F0912201908180915703892B8083809151
:104780004E038823D9F10E94A62420914C03309136
:104790004D038217930748F00E94A62420914C03F2
:1047A00030914D03821B930B0AC00E94A6242091D6
:1047B0004C0330914D0320953095820F931F8C321E
:1047C000914070F08091590380FF08C08AEC96E018
:1047D0009F938F930E949A070F900F900E949723A8
:1047E000E0912101F0912201908180914E03892B6B
:1047F00080830E949E2381110E9497238091210132
:10480000909122010C941E1890939B0180939A0121
:1048100008958295982F9C7C392F36953695282FB0
:10482000237344E0249FC0011124932F982B292F38
:104830002A7A2695892F8575880F822B08950895E9
:10484000CF93DF9300D000D01F92CDB7DEB70F908B
:104850000F900F900F900F90DF91CF9108950895D2
:1048600008950C948F1980916E03843021F1109279
:104870005A0320E488E190E00FB6F894A89580935D
:1048800060000FBE2093600083B7817F846083BF88
:1048900083B7816083BF7894889583B78E7F83BF09
:1048A0000FB6F894A89580916000886180936000AD
:1048B000109260000FBE0895CF930E94CA080E9414
:1048C000E1070E94CC08C0E08C2F0E94C108811132
:1048D00004C0CF5FC031C1F701C081E0CF9108951E
:1048E0000E9491190C94ED1D1F920F920FB60F921A
:1048F00011248F939F93AF93BF9380915A0381119B
:1049000013C080915B0390915C03A0915D03B09113
:104910005E034196A11DB11D80935B0390935C03E0
:10492000A0935D03B0935E03BF91AF919F918F9170
:104930000F900FBE0F901F90189582E084BD93E0FA
:1049400095BD9AEF97BD80936E0008952FB7F894A8
:1049500080915B0390915C03A0915D03B0915E0335
:104960002FBF08952FB7F89460915B0370915C039B
:1049700080915D0390915E032FBF0895CF92DF92E7
:10498000EF92FF920F931F932FB7F89440915B0320
:1049900050915C0360915D0370915E032FBF6A01CB
:1049A0007B01EE24FF248C0120E030E0C016D1060C
:1049B000E206F30610F4415051099A01281B390B05
:1049C000C9011F910F91FF90EF90DF90CF90089554
:1049D000CF92DF92EF92FF920F931F932FB7F8942D
:1049E000C0905B03D0905C03E0905D03F0905E03A9
:1049F0002FBF97018601061B170B280B390BC61614
:104A0000D706E806F90618F0C901B80106C0C901C1
:104A1000B80161507109810991091F910F91FF90AF
:104A2000EF90DF90CF9008951F920F920FB60F92E4
:104A300011248F939F93AF93BF9380915B039091C9
:104A40005C03A0915D03B0915E030196A11DB11DB1
:104A500080935B0390935C03A0935D03B0935E032C
:104A6000BF91AF919F918F910F900FBE0F901F90AC
:104A700018950E942615F8942FEF87EA91E62150A9
:104A800080409040E1F700C0000087E090EBDC013F
:104A90008093770390937803A0937903B0937A037C
:104AA0009CE088E10FB6F894A895809360000FBE53
:104AB00090936000FFCF28E0929FF0011124E80F4F
:104AC000F11DEE58FE4F9491892F8F7092959F7033
:104AD0000895CF93C82FCB010E945B25282F30E08B
:104AE00080E1989FA0011124422B532B403851059F
:104AF00019F480E090E015C09770E92FF0E088E0AD
:104B0000C89FE00DF11D112484E0EE0FFF1F8A9570
:104B1000E1F7E20FF31FEE0FFF1FE050F849859118
:104B20009491CF91089580E090E008950895809148
:104B3000610380FF0BC06091260185E0689FB00192
:104B4000112475956795759567952BC081FF09C0F0
:104B50006091260185E0689FB001112475956795E5
:104B600020C082FF07C06091260185E0689FB001E8
:104B7000112417C0909162039923D1F0609125010F
:104B8000961788F72091260185E0289F900111242F
:104B9000929FA001939F500D112470E0CA010E94C2
:104BA0005F2D6038710540F46115710539F002C060
:104BB00065E070E0862F08958FE7089581E00895FD
:104BC0008091610380FF08C06091240170E07595B9
:104BD00067957595679521C081FF06C06091240196
:104BE00070E07595679519C082FF04C0609124013B
:104BF00070E010C0909162039923C1F0609123018D
:104C00009617A0F780912401899FC001112470E0BC
:104C10000E945F2D6038710528F46115710521F03F
:104C2000862F08958FE7089581E0089561E070E090
:104C3000F4CF803F21F40E949725819504C0813FE5
:104C400029F40E949725809365030895823F21F4FB
:104C50000E949725819504C0833F29F40E949725DF
:104C6000809364030895893F19F40E94E02505C0EC
:104C70008A3F31F40E94E025819580936603089570
:104C80008B3F21F40E94E025819504C08C3F29F4DC
:104C90000E94E025809367030895843F21F480916A
:104CA0006303816017C0853F21F4809163038260B4
:104CB00011C0863F21F48091630384600BC0873F5D
:104CC00021F480916303886005C0883F31F48091AE
:104CD000630380618093630308958D3F21F4809185
:104CE000610381600BC08E3F21F48091610382607B
:104CF00005C08F3F29F48091610384608093610334
:104D00000895803F39F48091650387FF6CC010924D
:104D1000650369C0813F29F4809165031816BCF3CF
:104D200062C090916403823F29F497FF5CC01092A7
:104D3000640359C0833F19F41916CCF354C0893F5A
:104D400041F48091660318160CF04DC01092660372
:104D50004AC08A3F29F48091660387FF44C0F6CF9A
:104D60008B3F39F48091670387FF3DC01092670342
:104D70003AC08C3F29F4809167031816BCF333C006
:104D8000843F21F4809163038E7F17C0853F21F417
:104D9000809163038D7F11C0863F21F4809163036E
:104DA0008B7F0BC0873F21F480916303877F05C011
:104DB000883F31F4809163038F7E8093630313C037
:104DC0008D3F21F4809161038E7F0BC08E3F21F4D3
:104DD000809161038D7F05C08F3F29F4809161032D
:104DE0008B7F809361038091640381110EC0809159
:104DF000650381110AC080916603811106C080910C
:104E00006703811102C010926203089580915903D3
:104E100083FF7EC083E097E00E94010780916303D7
:104E20001F928F938EEF96E09F938F930E949A0725
:104E30008CEF96E00E94010780916403282F082ED2
:104E4000000C330B3F938F9389EF96E09F938F93E2
:104E50000E949A0787EF96E00E9401078091650300
:104E6000282F082E000C330B3F938F9384EF96E08E
:104E70009F938F930E949A0782EF96E00E9401070A
:104E800080916603282F082E000C330B3F938F93DD
:104E90008FEE96E09F938F930E949A078DEE96E097
:104EA0000E94010780916703282F082E000C330B06
:104EB0003F938F938AEE96E09F938F930E949A0779
:104EC00087EE96E00E940107809162031F928F9304
:104ED00084EE96E09F938F930E949A0782EE96E06D
:104EE0000E940107809161031F928F938FED96E0DE
:104EF0009F938F930E949A078CED96E00E94010782
:104F00008DB79EB74C960FB6F8949EBF0FBE8DBF5F
:104F100083E693E00E9467180E94A62490936003A2
:104F200080935F0308951F93CF93DF9380915F0376
:104F3000909160030E94BE24AC019091620399237A
:104F400021F02091270130E006C0209128018AE05D
:104F5000289F900111244217530708F485C08091BF
:104F60006403C0916503D0916603109167038111BA
:104F700007C0C11175C0D11173C0111171C074C0C7
:104F80009F3F19F09F5F90936203181624F40E94CC
:104F90009725809364038091640387FF05C00E9476
:104FA00097258195809364031C1624F40E9497250D
:104FB000809365038091650387FF05C00E94972554
:104FC00081958093650360916403662331F1C091FC
:104FD0006503CC2311F1062E000C770B880B990B7F
:104FE0000E94462C23E333E343E35FE30E94AA2CB1
:104FF0000E940E2C609364036C2FCC0F770B880BF0
:10500000990B0E94462C23E333E343E35FE30E94C2
:10501000AA2C0E940E2C609365031D1624F40E9496
:10502000E025809366038091660387FF05C00E9498
:10503000E025819580936603111624F40E94E025F3
:10504000809367038091670387FF05C00E94E02576
:10505000819580936703DF91CF911F910C94062770
:105060009F3F09F08FCF97CFDF91CF911F91089588
:10507000E3E6F3E085E0DF011D928A95E9F71092FF
:10508000620310926103089586E299E00E9401078D
:105090001F9281E08F931F9285E08F9388ED98E0B7
:1050A0009F938F930E949A070F900F900F900F90ED
:1050B0000F900F9008958330E9F128F4813061F06A
:1050C000823009F10895853009F462C008F449C0BE
:1050D000863009F474C0089580912801262F30E0AD
:1050E000280F311D2F3F310524F4680F60932801EC
:1050F00003C08FEF80932801809128011F928F9326
:1051000081E198E072C080912701262F30E0280FBE
:10511000311D2F3F310524F4680F6093270103C030
:105120008FEF80932701809127011F928F938FEF3C
:1051300097E05BC080912601262F30E0280F311DBB
:105140002F3F310524F4680F6093260103C08FEFD1
:1051500080932601809126011F928F938CEE97E019
:1051600044C080912501262F30E0280F311D2F3FAC
:10517000310524F4680F6093250103C08FEF8093FD
:105180002501809125011F928F9387ED97E02DC017
:1051900080912401262F30E0280F311D2F3F31054B
:1051A00024F4680F6093240103C08FEF80932401DF
:1051B000809124011F928F938EEB97E016C080910F
:1051C0002301262F30E0280F311D2F3F310524F415
:1051D000680F6093230103C08FEF809323018091B8
:1051E00023011F928F9383EA97E09F938F930E94EE
:1051F0009A070F900F900F900F900895833081F1D0
:1052000028F4813059F08230D1F00895853009F4C6
:1052100049C0B8F1863009F456C00895809128013C
:10522000681720F4861B8093280102C01092280181
:10523000809128011F928F9384E997E054C0809158
:105240002701681720F4861B8093270102C0109263
:105250002701809127011F928F9382E897E043C036
:1052600080912601681720F4861B8093260102C0D6
:1052700010922601809126011F928F938FE697E06E
:1052800032C080912501681720F4861B8093250188
:1052900002C010922501809125011F928F938AE50B
:1052A00097E021C080912401681720F4861B809329
:1052B000240102C010922401809124011F928F9337
:1052C00081E497E010C080912301681720F4861BC9
:1052D0008093230102C010922301809123011F9229
:1052E0008F9386E297E09F938F930E949A070F9087
:1052F0000F900F900F900895CF93C82F1F928F9308
:105300008BE29AE09F938F930E949A0781E090E04E
:10531000A0E0B0E0BC01CD0104C0660F771F881F7C
:10532000991FCA95D2F70E94FB210F900F900F9002
:105330000F90CF910C94ED1DCF93873288F58E316D
:1053400008F00BC18E3009F487C0D8F4873009F417
:1053500060C08B3009F44FC0863009F002C18091E3
:105360005903817F8E7F8093590380E39AE00E94E6
:10537000010785EE9CE00E94010781E080936903AC
:1053800046C0863109F4B0C020F4803109F47AC0F7
:10539000E8C0893109F491C08B3109F449C0E1C0FA
:1053A000883349F150F4893209F4D5C0853309F4C2
:1053B000D2C0873209F0D5C0CEC0833409F4CBC047
:1053C00028F48A3308F4CDC08953C8C0883409F062
:1053D000C8C00E94ED1D84ED9CE00E9401072FEFE4
:1053E00083ED90E3215080409040E1F700C0000041
:1053F0000E9439250CC087E59AE041C08BEB9CE008
:105400000E94010780915903816080935903C1E094
:10541000ADC080915903C82FC17080FFEFCF87ECDA
:105420009CE00E94010780915903817F8E7F3FC0DD
:105430009091590391FBCC27C0F981E0C827892FAF
:10544000C0FB81F980935903CC2319F08EEA9CE0CC
:1054500029C080EA9CE013C09091590392FBCC27AD
:10546000C0F981E0C827892FC0FB82F980935903D6
:10547000CC2319F081E99CE015C081E89CE00E94F2
:105480000107C5CF9091590393FBCC27C0F981E068
:10549000C827892FC0FB83F980935903CC2351F08F
:1054A00085E79CE00E940107809159038160809309
:1054B00059035CC088E69CE0E2CF89E59CE00E944D
:1054C00001078CE29CE00E94010785EF9BE00E94AF
:1054D000010788EC9BE00E94010783E89BE00E94A3
:1054E000010785E59BE0CBCF87E49BE00E940107A5
:1054F0000E9412181F928F938DE29BE09F938F93CF
:105500000E949A07809120011F928F9386E19BE071
:105510009F938F930E949A078091F4021F928F931A
:1055200083E09BE09F938F930E949A070E94B2248E
:105530009F938F937F936F938CEE9AE09F938F93BB
:105540000E949A078DB79EB742960FB6F8949EBFF9
:105550000FBE8DBF5CCF80E001C08D510E947C29C1
:1055600056CF8AEE9AE00E940107C0E08C2FCF91BF
:105570000895CF93C82F80916903813071F020F096
:10558000823009F44BC042C1E0912101F091220127
:105590008081823209F03CC107C0E0912101F09185
:1055A00022018081823261F48C2F0E94010C8111D2
:1055B00004C08C2F0E949C292FC081E090E02CC059
:1055C0008C2F0E942E0E811126C0C431E1F070F4A0
:1055D000CB3081F0C031D1F40E94442883E29AE0BC
:1055E0000E94010782E08093690315C0C93259F017
:1055F000C83361F480E39AE00E94010787E29AE0F1
:105600000E94010708C01092690304C181E29AE078
:105610000E940107FFC081E08170FEC0C43228F5FE
:10562000CE3108F0C1C0CB30A1F1D0F4C73009F0C1
:10563000D3C08EE18093280182E3809327018AE022
:105640008093260184E18093250188E080932401E2
:1056500088E28093230187EC98E00E940107BFC095
:10566000C33149F1C431C1F0B7C0CB3409F4A9C08A
:1056700028F4C93289F0C83361F0AEC0C13509F4ED
:105680009EC0C23509F499C0CE3409F0A5C06AE0C5
:105690009EC00E944428A3C080916803882319F00B
:1056A000109268039CC084ED98E00E94010781E09D
:1056B00080936903B1C08EEA98E00E9401078CE9EB
:1056C00098E00E940107809128011F928F9389E939
:1056D00098E09F938F930E949A0787E998E00E9431
:1056E000010785E898E00E940107809127011F9239
:1056F0008F9382E898E09F938F930E949A0780E8A7
:1057000098E00E94010781E798E00E9401078091DC
:1057100026011F928F938EE698E09F938F930E94AD
:105720009A078CE698E00E9401078BE598E00E94BA
:105730000107809125011F928F9388E598E09F9340
:105740008F930E949A0786E598E00E94010781E402
:1057500098E00E940107809124011F928F938EE3AD
:1057600098E09F938F930E949A078CE398E00E94A1
:10577000010785E298E00E940107809123011F92B2
:105780008F9382E298E09F938F930E949A0780E222
:1057900098E00E9401078DB79EB748960FB6F8941F
:1057A0009EBF0FBE8DBF1BC0CE51EC2FF0E0E05767
:1057B000FE4F80818093680312C061E003C061E006
:1057C00006C06AE0809168030E945B2808C080914F
:1057D00068030E94FE2803C085EC98E013C0809106
:1057E0006803882369F01F928F938FEB98E09F9353
:1057F0008F930E949A070F900F900F900F9004C004
:105800008CEB98E00E94010781E006C010926903CA
:1058100080E002C080E000CFCF9108950E94152C57
:105820006894B1110C94A42C08950E94892C88F0DE
:105830009F5798F0B92F9927B751B0F0E1F0660F54
:10584000771F881F991F1AF0BA95C9F714C0B13095
:1058500091F00E94A32CB1E008950C94A32C672F23
:10586000782F8827B85F39F0B93FCCF386957795C4
:105870006795B395D9F73EF49095809570956195AD
:105880007F4F8F4F9F4F0895E89409C097FB3EF4D8
:1058900090958095709561957F4F8F4F9F4F99237D
:1058A000A9F0F92F96E9BB279395F69587957795FB
:1058B0006795B795F111F8CFFAF4BB0F11F460FFBB
:1058C0001BC06F5F7F4F8F4F9F4F16C0882311F013
:1058D00096E911C0772321F09EE8872F762F05C027
:1058E000662371F096E8862F70E060E02AF09A95C2
:1058F000660F771F881FDAF7880F9695879597F9B7
:10590000089557FD9058440F551F59F05F3F71F0AF
:105910004795880F97FB991F61F09F3F79F0879516
:105920000895121613061406551FF2CF4695F1DF9F
:1059300008C0161617061806991FF1CF869571052F
:10594000610508940895E894BB2766277727CB0163
:1059500097F908950E94BD2C0C942E2D0E94202DA5
:1059600038F00E94272D20F0952311F00C94172D6C
:105970000C941D2D11240C94A42C0E94812C70F3E6
:10598000959FC1F3950F50E0551F629FF001729FE4
:10599000BB27F00DB11D639FAA27F00DB11DAA1FF3
:1059A000649F6627B00DA11D661F829F2227B00D40
:1059B000A11D621F739FB00DA11D621F839FA00DCB
:1059C000611D221F749F3327A00D611D231F849F1B
:1059D000600D211D822F762F6A2F11249F57504072
:1059E0009AF0F1F088234AF0EE0FFF1FBB1F661FED
:1059F000771F881F91505040A9F79E3F510580F0B6
:105A00000C94172D0C94A42C5F3FE4F3983ED4F330
:105A1000869577956795B795F795E7959F5FC1F759
:105A2000FE2B880F911D9695879597F9089597F904
:105A30009F6780E870E060E008959FEF80EC089534
:105A400000240A941616170618060906089500245D
:105A50000A9412161306140605060895092E0394D7
:105A6000000C11F4882352F0BB0F40F4BF2B11F44B
:105A700060FF04C06F5F7F4F8F4F9F4F0895991B4A
:105A800079E004C0991F961708F0961B881F7A9535
:105A9000C9F780950895AA1BBB1B51E107C0AA1F37
:105AA000BB1FA617B70710F0A61BB70B881F991FBF
:105AB0005A95A9F780959095BC01CD01089597FB63
:105AC000072E16F4009407D077FD09D00E944B2DC5
:105AD00007FC05D03EF4909581959F4F08957095F1
:105AE00061957F4F0895A1E21A2EAA1BBB1BFD01F1
:105AF0000DC0AA1FBB1FEE1FFF1FA217B307E407AD
:105B0000F50720F0A21BB30BE40BF50B661F771F04
:105B1000881F991F1A9469F76095709580959095E4
:105B20009B01AC01BD01CF010895EE0FFF1F059051
:0A5B3000F491E02D0994F894FFCFE2
:105B3A00560959095A095B095C095209D609BC096F
:105B4A0055095D090A01CB10BC1199116511311172
:105B5A00014F032808140A321E524E2D3432004CCB
:105B6A00554641004F4646004F4E00434F4E4E00A9
:105B7A00506F776572656400556E6174746163680D
:105B8A0065640044656661756C740041646472659D
:105B9A007373656400436F6E666967757265640046
:105BAA003F0053757370656E64656400404D36221C
:105BBA003206E505AF058D05190532054B05640565
:0A5BCA0001020304050607080900A4
:1068000088000000000000000400050006000700EA
:10681000080009000A000B000C000D000E000F001C
:1068200010001100120013001400150016001700CC
:10683000180019001A001B001C001D001E001F007C
:10684000200021002200230024002500260027002C
:10685000280035002A002B002C002D002E002F00D0
:1068600030000000320033003400290036003700C9
:106870003800E00000000000000000000000000000
:106880000000000000000000000000000000000008
:1068900000000000000000000000000000004F00A9
:1068A00050005100520000000000000000000000F5
:1068B00000000000000000000000000000000000D8
:1068C00000000000000000000000000000000000C8
:1068D00000000000000000000000000000000000B8
:1068E0000000000000000000890087008A008B0083
:1068F000F1A1E100E200E300F1A1E500E600000003
:106900000100000000000000EA4401000100E24430
:106910000100010001005500460054004A004B00F0
:10692000560057004700480001000100E9440100FB
:106930000100010001000100010001003A003B00DC
:106940003C003D003E003F0040004100420043004B
:10695000580001004C00390001004400450052007D
:1069600001000000010050004F0081404D004E002A
:1069700051000100000000000000000000000000C5
:106980000000000000000000000000000000000007
:1069900000000000000000000000000000004D00AA
:1069A0004A004E004B000000000000000000000004
:1069B00000000000000000000000000000000000D7
:1069C00000000000000000000000000000000000C7
:1069D00000000000000000000000000000000000B7
:1069E000000000000000000049000100010001005B
:1069F0000100010001000100010001000100000090
:00000001FF
